 sgx_render_flip_test

 Timestamp is 4be8cebd (Tue May 11 12:27:57 2010)

 Preferred load address is 00010000

 Start         Length     Name                   Class
 0001:00000000 00000004H .CRT$XCA                CODE
 0001:00000004 00000004H .CRT$XCZ                CODE
 0001:00000008 00000004H .CRT$XIA                CODE
 0001:0000000c 00000004H .CRT$XIZ                CODE
 0001:00000010 00000004H .CRT$XPA                CODE
 0001:00000014 00000004H .CRT$XPZ                CODE
 0001:00000018 00000004H .CRT$XTA                CODE
 0001:0000001c 00000004H .CRT$XTZ                CODE
 0001:00000020 00002ae3H .rdata                  CODE
 0001:00002b04 00000031H .rdata$debug            CODE
 0001:00002b38 00007360H .text                   CODE
 0001:00009e98 00000020H .xdata                  CODE
 0001:00009eb8 00000028H .idata$2                CODE
 0001:00009ee0 00000014H .idata$3                CODE
 0001:00009ef4 00000178H .idata$4                CODE
 0001:0000a06c 0000020cH .idata$6                CODE
 0001:0000a278 00000000H .edata                  CODE
 0002:00000000 00000178H .idata$5                DATA
 0002:00000178 0000001cH .data                   DATA
 0002:00000194 00000050H .bss                    DATA
 0003:00000000 000001a8H .pdata                  DATA

  Address         Publics by Value              Rva+Base       Lib:Object

 0000:00000000       ___safe_se_handler_count   00000000     <absolute>
 0000:00000000       ___safe_se_handler_table   00000000     <absolute>
 0001:00000000       __xc_a                     00011000     corelib0:crt0init.obj
 0001:00000004       __xc_z                     00011004     corelib0:crt0init.obj
 0001:00000008       __xi_a                     00011008     corelib0:crt0init.obj
 0001:0000000c       __xi_z                     0001100c     corelib0:crt0init.obj
 0001:00000010       __xp_a                     00011010     corelib0:crt0init.obj
 0001:00000014       __xp_z                     00011014     corelib0:crt0init.obj
 0001:00000018       __xt_a                     00011018     corelib0:crt0init.obj
 0001:0000001c       __xt_z                     0001101c     corelib0:crt0init.obj
 0001:0000003c       ??_C@_0P@NCGIOKND@No?5Sync?5Object?$AA@ 0001103c     sgx_render_flip_test.obj
 0001:0000004c       ??_C@_03MKLIJLBP@?9ns?$AA@ 0001104c     sgx_render_flip_test.obj
 0001:00000050       ??_C@_0BI@CLOENPIA@Render?5Context?5Priority?$AA@ 00011050     sgx_render_flip_test.obj
 0001:00000068       ??_C@_04KEBEIHMP@?9rcp?$AA@ 00011068     sgx_render_flip_test.obj
 0001:00000070       ??_C@_04CKDBHHCG@?9opr?$AA@ 00011070     sgx_render_flip_test.obj
 0001:00000078       ??_C@_0N@LANNGDHD@Verbose?5mode?$AA@ 00011078     sgx_render_flip_test.obj
 0001:00000088       ??_C@_02EJEOCNCO@?9v?$AA@  00011088     sgx_render_flip_test.obj
 0001:0000008c       ??_C@_04JMNPLBLF@?9dpa?$AA@ 0001108c     sgx_render_flip_test.obj
 0001:00000094       ??_C@_03INCBJOIL@?9ct?$AA@ 00011094     sgx_render_flip_test.obj
 0001:00000098       ??_C@_03JEPGDNNJ@?9db?$AA@ 00011098     sgx_render_flip_test.obj
 0001:0000009c       ??_C@_0CB@HGCMELHJ@Frequency?5of?5frame?5number?5output@ 0001109c     sgx_render_flip_test.obj
 0001:000000c0       ??_C@_03OJPDENCI@?9sf?$AA@ 000110c0     sgx_render_flip_test.obj
 0001:000000c4       ??_C@_04DAHOMCCH@?9phr?$AA@ 000110c4     sgx_render_flip_test.obj
 0001:000000cc       ??_C@_0CM@MJKCIIIE@Slow?5down?5factor?5for?53D?5hardware@ 000110cc     sgx_render_flip_test.obj
 0001:000000f8       ??_C@_04MCLDOKOJ@?9sd3?$AA@ 000110f8     sgx_render_flip_test.obj
 0001:00000100       ??_C@_0CM@PDLNPCEC@Slow?5down?5factor?5for?5TA?5hardware@ 00011100     sgx_render_flip_test.obj
 0001:0000012c       ??_C@_04HNILDDCL@?9sdt?$AA@ 0001112c     sgx_render_flip_test.obj
 0001:00000134       ??_C@_03PPELMDFC@?9mf?$AA@ 00011134     sgx_render_flip_test.obj
 0001:00000138       ??_C@_0CI@CAFEKBAA@Grid?5position?5to?5determine?5bound@ 00011138     sgx_render_flip_test.obj
 0001:00000160       ??_C@_03OOEEPDFD@?9gp?$AA@ 00011160     sgx_render_flip_test.obj
 0001:00000164       ??_C@_0CE@LBGOKMKP@Grid?5size?5to?5determine?5bounding?5@ 00011164     sgx_render_flip_test.obj
 0001:00000188       ??_C@_03MFGJKAJA@?9gs?$AA@ 00011188     sgx_render_flip_test.obj
 0001:0000018c       ??_C@_0CE@CPFGKJII@Multithreaded?5with?5grid?5size?5?$CIx?0@ 0001118c     sgx_render_flip_test.obj
 0001:000001b0       ??_C@_07LPJCHBPO@?$HLx?$HN?5?$HLy?$HN?$AA@ 000111b0     sgx_render_flip_test.obj
 0001:000001b8       ??_C@_03IHLPLDIB@?9mt?$AA@ 000111b8     sgx_render_flip_test.obj
 0001:000001bc       ??_C@_0BM@OGGOLKGL@Use?5present?5blit?5?$CIsoftware?$CJ?$AA@ 000111bc     sgx_render_flip_test.obj
 0001:000001d8       ??_C@_03MDKCGCHL@?9bs?$AA@ 000111d8     sgx_render_flip_test.obj
 0001:000001dc       ??_C@_0BL@EMDAHIMJ@Use?5present?5blit?5?$CI2D?5core?$CJ?$AA@ 000111dc     sgx_render_flip_test.obj
 0001:000001f8       ??_C@_03CKMABMDP@?9b2?$AA@ 000111f8     sgx_render_flip_test.obj
 0001:000001fc       ??_C@_0BB@NOOLFKLF@Use?5present?5blit?$AA@ 000111fc     sgx_render_flip_test.obj
 0001:00000210       ??_C@_02GHOAPKHL@?9b?$AA@  00011210     sgx_render_flip_test.obj
 0001:00000214       ??_C@_03NDKDKKFO@?9nr?$AA@ 00011214     sgx_render_flip_test.obj
 0001:00000218       ??_C@_03IFPJANNI@?9nt?$AA@ 00011218     sgx_render_flip_test.obj
 0001:0000021c       ??_C@_0M@LLDBDGHB@No?5flipping?$AA@ 0001121c     sgx_render_flip_test.obj
 0001:00000228       ??_C@_01GPOEFGEJ@?7?$AA@   00011228     sgx_render_flip_test.obj
 0001:0000022c       ??_C@_03PNANHNAL@?9nf?$AA@ 0001122c     sgx_render_flip_test.obj
 0001:00000230       ??_C@_03IAHKIJEO@?9nc?$AA@ 00011230     sgx_render_flip_test.obj
 0001:00000234       ??_C@_03KONEFOBL@?9nw?$AA@ 00011234     sgx_render_flip_test.obj
 0001:00000238       ??_C@_02NCEOIEDG@?9o?$AA@  00011238     sgx_render_flip_test.obj
 0001:0000023c       ??_C@_04LCKJFJBK@?9hwr?$AA@ 0001123c     sgx_render_flip_test.obj
 0001:00000244       ??_C@_04HHAMBNME@?9neo?$AA@ 00011244     sgx_render_flip_test.obj
 0001:0000024c       ??_C@_0CH@EHPOEMFN@Number?5of?5frames?5per?5triangle?5ro@ 0001124c     sgx_render_flip_test.obj
 0001:00000274       ??_C@_04FHDJDIKM@?9fpr?$AA@ 00011274     sgx_render_flip_test.obj
 0001:0000027c       ??_C@_03JJGBLIAP@?9nb?$AA@ 0001127c     sgx_render_flip_test.obj
 0001:00000280       ??_C@_0BM@HFNLMCFM@Background?5colour?5in?5RGB888?$AA@ 00011280     sgx_render_flip_test.obj
 0001:0000029c       ??_C@_03IJGAHACK@?9bc?$AA@ 0001129c     sgx_render_flip_test.obj
 0001:000002a0       ??_C@_0EA@COCGJEHO@Triangle?5Vertex?5Colour?53?5in?5RGB8@ 000112a0     sgx_render_flip_test.obj
 0001:000002e0       ??_C@_04PACCAMFO@?9vc3?$AA@ 000112e0     sgx_render_flip_test.obj
 0001:000002e8       ??_C@_0DP@BNANPDBO@Triangle?5Vertex?5Colour?52?5in?5RGB8@ 000112e8     sgx_render_flip_test.obj
 0001:00000328       ??_C@_03KCPGDJCN@?$HLx?$HN?$AA@ 00011328     sgx_render_flip_test.obj
 0001:0000032c       ??_C@_04OJDJDNBP@?9vc2?$AA@ 0001132c     sgx_render_flip_test.obj
 0001:00000334       ??_C@_0CB@CAODBHAH@Triangle?5Vertex?5Colour?5in?5RGB888@ 00011334     sgx_render_flip_test.obj
 0001:00000358       ??_C@_04JELPBBAF@?$HLx?$HN?7?$AA@ 00011358     sgx_render_flip_test.obj
 0001:00000360       ??_C@_03JCEPHLIG@?9vc?$AA@ 00011360     sgx_render_flip_test.obj
 0001:00000364       ??_C@_0BO@CAPDADMG@Number?5of?5Triangles?5per?5frame?$AA@ 00011364     sgx_render_flip_test.obj
 0001:00000384       ??_C@_04IDIHHAON@?9tpf?$AA@ 00011384     sgx_render_flip_test.obj
 0001:0000038c       ??_C@_0P@IBJMDFC@Triangle?5Style?$AA@ 0001138c     sgx_render_flip_test.obj
 0001:0000039c       ??_C@_03NLAJLNLJ@?9ts?$AA@ 0001139c     sgx_render_flip_test.obj
 0001:000003a0       ??_C@_0CA@KDDMHPJK@Message?5to?5display?5when?5pausing?$AA@ 000113a0     sgx_render_flip_test.obj
 0001:000003c0       ??_C@_04EDLOJGAE@?$HLs?$HN?7?$AA@ 000113c0     sgx_render_flip_test.obj
 0001:000003c8       ??_C@_03IEBCKLK@?9pm?$AA@  000113c8     sgx_render_flip_test.obj
 0001:000003cc       ??_C@_0CH@GPAABPOI@Pause?5?$CIwait?5for?5user?$CJ?5every?5?8n?8?5@ 000113cc     sgx_render_flip_test.obj
 0001:000003f4       ??_C@_02BPBEIKKI@?9p?$AA@  000113f4     sgx_render_flip_test.obj
 0001:000003f8       ??_C@_0BN@DMBIAPHB@Dump?5bitmap?5every?5?8n?8?5frames?$AA@ 000113f8     sgx_render_flip_test.obj
 0001:00000418       ??_C@_04POJDPNFK@?9bmp?$AA@ 00011418     sgx_render_flip_test.obj
 0001:00000420       ??_C@_0CN@GCCHICGB@Serialise?5?$CIwait?5for?5render?$CJ?5ever@ 00011420     sgx_render_flip_test.obj
 0001:00000450       ??_C@_03LKFNOGOP@?$HLn?$HN?$AA@ 00011450     sgx_render_flip_test.obj
 0001:00000454       ??_C@_04CKBDPOJK@?9ser?$AA@ 00011454     sgx_render_flip_test.obj
 0001:0000045c       ??_C@_04OHKKDBIB@?9us2?$AA@ 0001145c     sgx_render_flip_test.obj
 0001:00000464       ??_C@_03NKMLNHIO@?9us?$AA@ 00011464     sgx_render_flip_test.obj
 0001:00000468       ??_C@_0BM@DEHLBJOE@Sleep?5between?5renders?5in?5ms?$AA@ 00011468     sgx_render_flip_test.obj
 0001:00000484       ??_C@_04NOGJKOLN@?$HLt?$HN?7?$AA@ 00011484     sgx_render_flip_test.obj
 0001:0000048c       ??_C@_02DEDJNJGL@?9s?$AA@  0001148c     sgx_render_flip_test.obj
 0001:00000490       ??_C@_0BN@MOCIGDHE@Parameter?5Buffer?5size?5in?5KiB?$AA@ 00011490     sgx_render_flip_test.obj
 0001:000004b0       ??_C@_03IPNJDGHF@?9pb?$AA@ 000114b0     sgx_render_flip_test.obj
 0001:000004b4       ??_C@_0BG@LDGJAOMH@Starting?5frame?5number?$AA@ 000114b4     sgx_render_flip_test.obj
 0001:000004cc       ??_C@_03MEKLMKKH@?9fs?$AA@ 000114cc     sgx_render_flip_test.obj
 0001:000004d0       ??_C@_0CB@NKMBLHFN@Total?5number?5of?5frames?5to?5render@ 000114d0     sgx_render_flip_test.obj
 0001:000004f4       ??_C@_02DIMDPHP@?9f?$AA@   000114f4     sgx_render_flip_test.obj
 0001:000004f8       ??_C@_0BN@GFAMLLDC@Swap?5interval?5for?5flip?5chain?$AA@ 000114f8     sgx_render_flip_test.obj
 0001:00000518       ??_C@_04OBMNBJEG@?$HLn?$HN?7?$AA@ 00011518     sgx_render_flip_test.obj
 0001:00000520       ??_C@_03GOGLFBOH@?9si?$AA@ 00011520     sgx_render_flip_test.obj
 0001:00000a60       ??_C@_0BA@GHGHGFGN@Primary?5Surface?$AA@ 00011a60     sgx_render_flip_test.obj
 0001:00000a70       ??_C@_0M@PMHHPIHO@Swap?5Buffer?$AA@ 00011a70     sgx_render_flip_test.obj
 0001:00000a7c       ??_C@_0M@MIFEGCGI@Back?5buffer?$AA@ 00011a7c     sgx_render_flip_test.obj
 0001:00000a88       ??_C@_0CE@FOADKLNF@waiting?5for?5renders?5to?5complete?4@ 00011a88     sgx_render_flip_test.obj
 0001:00000aac       ??_C@_0BJ@JIBJLILC@0x?$CFlx?3?5EOT?5USSE?5Program?6?$AA@ 00011aac     sgx_render_flip_test.obj
 0001:00000ac8       ??_C@_0BJ@MLIINBFG@0x?$CFlx?3?5EOR?5USSE?5Program?6?$AA@ 00011ac8     sgx_render_flip_test.obj
 0001:00000ae4       ??_C@_0BJ@EMCIPEDF@0x?$CFlx?3?5EOP?5USSE?5Program?6?$AA@ 00011ae4     sgx_render_flip_test.obj
 0001:00000b00       ??_C@_0CB@IHGKAJGH@0x?$CFlx?3?5Pixel?5Event?5PDS?5Program?6?6@ 00011b00     sgx_render_flip_test.obj
 0001:00000b24       ??_C@_0CE@LLJHEHPA@0x?$CFlx?3?5Secondary?5PDS?5Pixel?5Progr@ 00011b24     sgx_render_flip_test.obj
 0001:00000b48       ??_C@_0CF@GDIAKAOK@0x?$CFlx?3?5Secondary?5USSE?5Pixel?5Prog@ 00011b48     sgx_render_flip_test.obj
 0001:00000b70       ??_C@_0BN@IDFCOLNP@0x?$CFlx?3?5?$CFs?5Pixel?5PDS?5Program?6?$AA@ 00011b70     sgx_render_flip_test.obj
 0001:00000b90       ??_C@_0BO@HNFONIPG@0x?$CFlx?3?5?$CFs?5Pixel?5USSE?5Program?6?$AA@ 00011b90     sgx_render_flip_test.obj
 0001:00000bb0       ??_C@_0CE@PKHOFDIJ@?60x?$CFlx?3?5MTE?5state?5copy?5PDS?5Progr@ 00011bb0     sgx_render_flip_test.obj
 0001:00000bd4       ??_C@_0CE@LHHPEIDP@0x?$CFlx?3?5MTE?5state?5copy?5USSE?5Progr@ 00011bd4     sgx_render_flip_test.obj
 0001:00000bf8       ??_C@_0CC@PPMIGHNH@0x?$CFlx?3?5Vertex?5shader?5PDS?5Program@ 00011bf8     sgx_render_flip_test.obj
 0001:00000c1c       ??_C@_0CD@HDPJMKEI@0x?$CFlx?3?5Vertex?5shader?5USSE?5Progra@ 00011c1c     sgx_render_flip_test.obj
 0001:00000c40       ??_C@_0BO@POIGAKIM@0x?$CFlx?3?5Terminate?5PDS?5Program?6?$AA@ 00011c40     sgx_render_flip_test.obj
 0001:00000c60       ??_C@_0CA@OINHEANG@0x?$CFlx?3?5Terminate?5USSE?5Program?6?6?$AA@ 00011c60     sgx_render_flip_test.obj
 0001:00000c80       ??_C@_0CN@DNMHKJMP@Adding?5render?5target?5via?5SGXAddR@ 00011c80     sgx_render_flip_test.obj
 0001:00000cb0       ??_C@_0BM@FKFLDJHI@Mean?5time?5per?5frame?3?5?$CFluus?6?$AA@ 00011cb0     sgx_render_flip_test.obj
 0001:00000ccc       ??_C@_01EEMJAFIK@?6?$AA@   00011ccc     sgx_render_flip_test.obj
 0001:00000cd0       ??_C@_0BD@FOJPDKHP@Total?5time?3?5?$CFlums?6?$AA@ 00011cd0     sgx_render_flip_test.obj
 0001:00000ce4       ??_C@_0CC@FHJCCNNC@Attempt?5to?5remove?5render?5target?3@ 00011ce4     sgx_render_flip_test.obj
 0001:00000d08       ??_C@_03OFAPEBGM@?$CFs?6?$AA@ 00011d08     sgx_render_flip_test.obj
 0001:00000d0c       ??_C@_0BC@GIBLDJKM@Background?5object?$AA@ 00011d0c     sgx_render_flip_test.obj
 0001:00000d20       ??_C@_08NMAPBDDP@Triangle?$AA@ 00011d20     sgx_render_flip_test.obj
 0001:00000d2c       ??_C@_0BE@KAGKHHLA@?$CFsFrame?5number?5?$CFlu?6?$AA@ 00011d2c     sgx_render_flip_test.obj
 0001:00000d40       ??_C@_0BM@HJEKHOOM@Allocate?5PB?5reserve?5memory?6?$AA@ 00011d40     sgx_render_flip_test.obj
 0001:00000d5c       ??_C@_0CN@BKDFEMBM@Allocate?5a?5static?5Fragment?5PDS?5b@ 00011d5c     sgx_render_flip_test.obj
 0001:00000d8c       ??_C@_0CL@OBMOGECF@Allocate?5a?5static?5Vertex?5PDS?5buf@ 00011d8c     sgx_render_flip_test.obj
 0001:00000db8       ??_C@_0CH@DDNMFBMM@Allocate?5a?5static?5vertex?5buffer?5@ 00011db8     sgx_render_flip_test.obj
 0001:00000de0       ??_C@_0CG@BNFOHFHJ@Allocate?5a?5static?5index?5buffer?5?$CI@ 00011de0     sgx_render_flip_test.obj
 0001:00000e08       ??_C@_0DD@HJPLJIBC@Allocate?5a?5static?5VDM?5control?5st@ 00011e08     sgx_render_flip_test.obj
 0001:00000e3c       ??_C@_0DA@CELKAMLC@Allocate?5a?5static?5vertex?5USE?5cod@ 00011e3c     sgx_render_flip_test.obj
 0001:00000e6c       ??_C@_0DC@HILOFAAF@Allocate?5a?5static?5fragment?5USE?5c@ 00011e6c     sgx_render_flip_test.obj
 0001:00000ea0       ??_C@_0BK@CMJKEHGE@Allocate?5back?5buffer?5?$CFlu?6?$AA@ 00011ea0     sgx_render_flip_test.obj
 0001:00000ebc       ??_C@_0CA@DGGJNKGO@?5Test?5Memory?5Allocation?5FAILED?6?$AA@ 00011ebc     sgx_render_flip_test.obj
 0001:00000edc       ??_C@_0M@IIANJMEI@?$CI?$CFlu?0?5?$CFlu?$CJ?5?$AA@ 00011edc     sgx_render_flip_test.obj
 0001:00000ee8       ??_C@_0DF@JJFELGBI@Please?5disable?5flipping?5when?5usi@ 00011ee8     sgx_render_flip_test.obj
 0001:00000f20       ??_C@_0CM@FEMEHKNK@Unexpected?5error?5parsing?5command@ 00011f20     sgx_render_flip_test.obj
 0001:00000f4c       ??_C@_0BO@GJABOMGM@Invalid?5status?5frequency?5?$CFlu?6?$AA@ 00011f4c     sgx_render_flip_test.obj
 0001:00000f6c       ??_C@_0CF@HLMNOFCM@Unknown?5memory?5flags?5test?5option@ 00011f6c     sgx_render_flip_test.obj
 0001:00000f94       ??_C@_0CE@IFHENFB@Unknown?5memory?5flags?5test?5value?5@ 00011f94     sgx_render_flip_test.obj
 0001:00000fb8       ??_C@_0CB@HCADHGDN@Memory?5flags?5test?5?$CIPDS?5Vertex?$CJ?3?5@ 00011fb8     sgx_render_flip_test.obj
 0001:00000fdc       ??_C@_0CA@KHNMJHPP@Memory?5flags?5test?5?$CIPDS?5Pixel?$CJ?3?5?$AA@ 00011fdc     sgx_render_flip_test.obj
 0001:00000ffc       ??_C@_0BI@HBNNBDGK@Not?5currently?5supported?$AA@ 00011ffc     sgx_render_flip_test.obj
 0001:00001014       ??_C@_0BJ@IMDICGNH@Invalid?5grid?5pos?5Y?3?5?$CFlu?6?$AA@ 00012014     sgx_render_flip_test.obj
 0001:00001030       ??_C@_0BJ@EAJCCGEJ@Invalid?5grid?5pos?5X?3?5?$CFlu?6?$AA@ 00012030     sgx_render_flip_test.obj
 0001:0000104c       ??_C@_0BK@FKFCBDB@Invalid?5grid?5size?5Y?3?5?$CFlu?6?$AA@ 0001204c     sgx_render_flip_test.obj
 0001:00001068       ??_C@_0BK@MJAPCBKP@Invalid?5grid?5size?5X?3?5?$CFlu?6?$AA@ 00012068     sgx_render_flip_test.obj
 0001:00001084       ??_C@_0BN@KIKPLJHG@Invalid?5MT?5grid?5size?5Y?3?5?$CFlu?6?$AA@ 00012084     sgx_render_flip_test.obj
 0001:000010a4       ??_C@_0BN@EEGLAPBH@Invalid?5grid?5MT?5size?5X?3?5?$CFlu?6?$AA@ 000120a4     sgx_render_flip_test.obj
 0001:000010c4       ??_C@_0CI@LCNOLPGA@2D?5core?5not?5supported?5on?5this?5pl@ 000120c4     sgx_render_flip_test.obj
 0001:000010ec       ??_C@_0BH@JHEOIMKN@Unknown?5hwr?5option?5?$CFs?6?$AA@ 000120ec     sgx_render_flip_test.obj
 0001:00001104       ??_C@_0BN@LCFEPEPL@Invalid?5triangle?5style?3?5?$CFlu?6?$AA@ 00012104     sgx_render_flip_test.obj
 0001:00001124       ??_C@_0DN@ECNCANJG@Swap?5interval?5should?5be?5below?525@ 00012124     sgx_render_flip_test.obj
 0001:00001164       ??_C@_0BN@EEGCGIOA@No?5SyncObject?5mode?3?5ENABLED?6?$AA@ 00012164     sgx_render_flip_test.obj
 0001:00001184       ??_C@_0BN@EMFDIKLK@Render?5Context?5Priority?3?5?$CFu?6?$AA@ 00012184     sgx_render_flip_test.obj
 0001:000011a4       ??_C@_0BK@DOKEHCGI@Output?5preamble?3?5ENABLED?6?$AA@ 000121a4     sgx_render_flip_test.obj
 0001:000011c0       ??_C@_0BH@PECOCMDD@Verbose?5mode?3?5ENABLED?6?$AA@ 000121c0     sgx_render_flip_test.obj
 0001:000011d8       ??_C@_0CC@MAAMACBB@Debug?5Program?5Addresses?3?5ENABLED@ 000121d8     sgx_render_flip_test.obj
 0001:000011fc       ??_C@_0BF@DEHIKBAB@Crash?5Test?3?5ENABLED?6?$AA@ 000121fc     sgx_render_flip_test.obj
 0001:00001214       ??_C@_0BG@BAPHFKJO@Debug?5Break?3?5ENABLED?6?$AA@ 00012214     sgx_render_flip_test.obj
 0001:0000122c       ??_C@_0BH@IKEIEIHN@Status?5frequency?3?5?$CFlu?6?$AA@ 0001222c     sgx_render_flip_test.obj
 0001:00001244       ??_C@_0CF@ENMKENDI@Parameters?5heap?5reserve?5factor?3?5@ 00012244     sgx_render_flip_test.obj
 0001:0000126c       ??_C@_0BJ@NOPOGOKJ@3D?5Slowdown?5Factor?3?5?$CFlu?6?$AA@ 0001226c     sgx_render_flip_test.obj
 0001:00001288       ??_C@_0BJ@PDIOLMFM@TA?5Slowdown?5Factor?3?5?$CFlu?6?$AA@ 00012288     sgx_render_flip_test.obj
 0001:000012a4       ??_C@_0N@JBABOGPP@EDM_PROTECT?5?$AA@ 000122a4     sgx_render_flip_test.obj
 0001:000012b4       ??_C@_05HGJNIKF@Read?5?$AA@ 000122b4     sgx_render_flip_test.obj
 0001:000012bc       ??_C@_06GJOMFEOM@Write?5?$AA@ 000122bc     sgx_render_flip_test.obj
 0001:000012c4       ??_C@_0CH@JBDEBGIH@Memory?5flags?5test?5?$CIUSSE?5Vertex?5C@ 000122c4     sgx_render_flip_test.obj
 0001:000012ec       ??_C@_03JMPGFMML@uvc?$AA@  000122ec     sgx_render_flip_test.obj
 0001:000012f0       ??_C@_0CC@POIFGBNN@Memory?5flags?5test?5?$CIUSSE?5Vertex?$CJ?3@ 000122f0     sgx_render_flip_test.obj
 0001:00001314       ??_C@_02CLOBFCCG@uv?$AA@   00012314     sgx_render_flip_test.obj
 0001:00001318       ??_C@_0CG@MHONNELB@Memory?5flags?5test?5?$CIUSSE?5Pixel?5Co@ 00012318     sgx_render_flip_test.obj
 0001:00001340       ??_C@_03JIHLCAHJ@upc?$AA@  00012340     sgx_render_flip_test.obj
 0001:00001344       ??_C@_0CB@PCLHIEKB@Memory?5flags?5test?5?$CIUSSE?5Pixel?$CJ?3?5@ 00012344     sgx_render_flip_test.obj
 0001:00001368       ??_C@_02HNLLPFKA@up?$AA@   00012368     sgx_render_flip_test.obj
 0001:0000136c       ??_C@_0CG@GKAAOAL@Memory?5flags?5test?5?$CIPDS?5Vertex?5Co@ 0001236c     sgx_render_flip_test.obj
 0001:00001394       ??_C@_05EOILKBOE@pdsvc?$AA@ 00012394     sgx_render_flip_test.obj
 0001:0000139c       ??_C@_04FLJJIAAA@pdsv?$AA@ 0001239c     sgx_render_flip_test.obj
 0001:000013a4       ??_C@_0CF@IBCMNALK@Memory?5flags?5test?5?$CIPDS?5Pixel?5Cod@ 000123a4     sgx_render_flip_test.obj
 0001:000013cc       ??_C@_05EKAGNNFG@pdspc?$AA@ 000123cc     sgx_render_flip_test.obj
 0001:000013d4       ??_C@_04NMDCHIG@pdsp?$AA@  000123d4     sgx_render_flip_test.obj
 0001:000013dc       ??_C@_0BK@KEMHMCF@Memory?5flags?5test?5?$CIPBE?$CJ?3?5?$AA@ 000123dc     sgx_render_flip_test.obj
 0001:000013f8       ??_C@_0BG@FBLPDCBG@Grid?5pos?3?5?$CI?$CFlu?0?5?$CFlu?$CJ?6?$AA@ 000123f8     sgx_render_flip_test.obj
 0001:00001410       ??_C@_0BG@NEABAIKF@Grid?5size?3?5?$CFlu?5x?5?$CFlu?6?$AA@ 00012410     sgx_render_flip_test.obj
 0001:00001428       ??_C@_0CC@LDNJFOHF@Multithread?5Grid?5size?3?5?$CFlu?5x?5?$CFlu@ 00012428     sgx_render_flip_test.obj
 0001:00001450       ??_C@_0EE@IMEGLFGG@WARNING?3?5Pthreads?5not?5supported?5@ 00012450     sgx_render_flip_test.obj
 0001:00001494       ??_C@_0BO@MLEBADMC@Blitting?5?$CIsoftware?$CJ?3?5ENABLED?6?$AA@ 00012494     sgx_render_flip_test.obj
 0001:000014b4       ??_C@_0BD@MJNKFODF@Blitting?3?5ENABLED?6?$AA@ 000124b4     sgx_render_flip_test.obj
 0001:000014c8       ??_C@_0BC@NHBAANIG@Render?3?5DISABLED?6?$AA@ 000124c8     sgx_render_flip_test.obj
 0001:000014dc       ??_C@_0BE@EDHFPOON@Transfer?3?5DISABLED?6?$AA@ 000124dc     sgx_render_flip_test.obj
 0001:000014f0       ??_C@_0BE@DEDGJIHE@Flipping?3?5DISABLED?6?$AA@ 000124f0     sgx_render_flip_test.obj
 0001:00001504       ??_C@_0CD@DCLBFHBM@Clean?5up?5at?5end?5of?5test?3?5DISABLE@ 00012504     sgx_render_flip_test.obj
 0001:00001528       ??_C@_0CM@GHGDDGJA@Wait?5for?5sync?5ops?5at?5end?5of?5test@ 00012528     sgx_render_flip_test.obj
 0001:00001554       ??_C@_0BA@JLDJLNAP@Overdraws?3?5?$CFlu?6?$AA@ 00012554     sgx_render_flip_test.obj
 0001:00001564       ??_C@_0CF@MJLEFGGD@Simulated?5?$CFs?5lockup?5every?5?$CFlu?5ki@ 00012564     sgx_render_flip_test.obj
 0001:0000158c       ??_C@_0O@KDBNMAOP@Pixel?5Backend?$AA@ 0001258c     sgx_render_flip_test.obj
 0001:0000159c       ??_C@_03OGFNAAND@pbe?$AA@  0001259c     sgx_render_flip_test.obj
 0001:000015a0       ??_C@_0N@MJGNOGPK@Pixel?5Shader?$AA@ 000125a0     sgx_render_flip_test.obj
 0001:000015b0       ??_C@_02FAFNGEII@ps?$AA@   000125b0     sgx_render_flip_test.obj
 0001:000015b4       ??_C@_0O@FEIBMPOA@Vertex?5Shader?$AA@ 000125b4     sgx_render_flip_test.obj
 0001:000015c4       ??_C@_02FENABIDK@vs?$AA@   000125c4     sgx_render_flip_test.obj
 0001:000015c8       ??_C@_03CJJGEMJ@VDM?$AA@   000125c8     sgx_render_flip_test.obj
 0001:000015cc       ??_C@_03PGCKJLF@vdm?$AA@   000125cc     sgx_render_flip_test.obj
 0001:000015d0       ??_C@_0BI@OAMAOACM@Event?5Object?3?5DISABLED?6?$AA@ 000125d0     sgx_render_flip_test.obj
 0001:000015e8       ??_C@_0CN@OFMEABGE@Number?5of?5frames?5per?5triangle?5ro@ 000125e8     sgx_render_flip_test.obj
 0001:00001618       ??_C@_0BK@EEHOCEJI@Number?5of?5buffers?3?50x?$CFlx?6?$AA@ 00012618     sgx_render_flip_test.obj
 0001:00001634       ??_C@_0BK@KOKIEJIN@Background?5Colour?3?50x?$CFlx?6?$AA@ 00012634     sgx_render_flip_test.obj
 0001:00001650       ??_C@_0BK@NIPCFHCI@Vertex?5Colour?5?$CI3?$CJ?3?50x?$CFlx?6?$AA@ 00012650     sgx_render_flip_test.obj
 0001:0000166c       ??_C@_0BK@BJHMIIOI@Vertex?5Colour?5?$CI2?$CJ?3?50x?$CFlx?6?$AA@ 0001266c     sgx_render_flip_test.obj
 0001:00001688       ??_C@_0BG@MNLKGKAI@Vertex?5Colour?3?50x?$CFlx?6?$AA@ 00012688     sgx_render_flip_test.obj
 0001:000016a0       ??_C@_0CE@HIOBJNLF@Number?5of?5triangles?5per?5frame?3?5?$CF@ 000126a0     sgx_render_flip_test.obj
 0001:000016c4       ??_C@_0BF@PHLPMHG@Triangle?5style?3?5?$CFlu?6?$AA@ 000126c4     sgx_render_flip_test.obj
 0001:000016dc       ??_C@_0BH@EJOHJHNL@?$CI?$CFs?$CJ?5?$DM?9?5Pause?5message?6?$AA@ 000126dc     sgx_render_flip_test.obj
 0001:000016f4       ??_C@_0BI@LFIDFLOJ@Pause?5every?5?$CFlu?5frames?6?$AA@ 000126f4     sgx_render_flip_test.obj
 0001:0000170c       ??_C@_0BJ@OINGDDNN@Bitmap?5every?5?$CFlu?5frames?6?$AA@ 0001270c     sgx_render_flip_test.obj
 0001:00001728       ??_C@_0BM@FCMEPIHF@Serialise?5every?5?$CFlu?5frames?6?$AA@ 00012728     sgx_render_flip_test.obj
 0001:00001744       ??_C@_0CK@MBJOKNLF@Microsecond?5sleep?5between?5kicks?5@ 00012744     sgx_render_flip_test.obj
 0001:00001770       ??_C@_0CK@PIBDJBHA@Microsecond?5sleep?5between?5kicks?5@ 00012770     sgx_render_flip_test.obj
 0001:0000179c       ??_C@_0BM@GLNPOGCM@Sleep?5between?5kicks?3?5?$CFlums?6?$AA@ 0001279c     sgx_render_flip_test.obj
 0001:000017b8       ??_C@_0CE@BFEJAGD@Parameter?5Buffer?5size?3?50x?$CFlx?5Byt@ 000127b8     sgx_render_flip_test.obj
 0001:000017dc       ??_C@_0BF@DMCADLEH@Starting?5frame?3?5?$CFlu?6?$AA@ 000127dc     sgx_render_flip_test.obj
 0001:000017f4       ??_C@_0BH@HKNNJNOG@Number?5of?5frames?3?5?$CFlu?6?$AA@ 000127f4     sgx_render_flip_test.obj
 0001:0000180c       ??_C@_0BE@LINCBDNC@Swap?5Interval?3?5?$CFlu?6?$AA@ 0001280c     sgx_render_flip_test.obj
 0001:00001820       ??_C@_0P@NONGIECF@Press?5ENTER?4?4?4?$AA@ 00012820     sgx_render_flip_test.obj
 0001:00001830       ??_C@_0DD@GODBIEMM@Display?5Class?5API?3?5unmap?5display@ 00012830     sgx_render_flip_test.obj
 0001:00001864       ??_C@_0BM@GKACHJHD@Destroy?5Primary?5Swap?5Chain?6?$AA@ 00012864     sgx_render_flip_test.obj
 0001:00001880       ??_C@_0EO@CKGGAHCN@Display?5Class?5API?3?5unmap?5swapcha@ 00012880     sgx_render_flip_test.obj
 0001:000018d0       ??_C@_0BP@GJLKNMBD@Destroy?5the?5transfer?5context?3?6?$AA@ 000128d0     sgx_render_flip_test.obj
 0001:000018f0       ??_C@_0CE@CHFCNMEA@Attempt?5to?5destroy?5render?5contex@ 000128f0     sgx_render_flip_test.obj
 0001:00001914       ??_C@_0CE@LAPEIHHC@No?5cleanup?5was?5specified?4?5Exitin@ 00012914     sgx_render_flip_test.obj
 0001:00001938       ??_C@_0BL@IPHOGMNB@Joining?5thread?5?$CI?$CFlu?0?5?$CFlu?$CJ?6?$AA@ 00012938     sgx_render_flip_test.obj
 0001:00001954       ??_C@_0BM@ECPPFIHB@Creating?5thread?5?$CI?$CFlu?0?5?$CFlu?$CJ?6?$AA@ 00012954     sgx_render_flip_test.obj
 0001:00001970       ??_C@_0DE@FNLBOPCP@Creating?5render?5context?5via?5SGXC@ 00012970     sgx_render_flip_test.obj
 0001:000019a8       ??_C@_0EE@CHBJKHJA@Attempt?5to?5set?5priority?5of?5trans@ 000129a8     sgx_render_flip_test.obj
 0001:000019ec       ??_C@_0DN@DENCIAJK@Priority?5of?5transfer?1render?5cont@ 000129ec     sgx_render_flip_test.obj
 0001:00001a2c       ??_C@_0BD@OEAFCFPL@Getting?5Misc?5Info?6?$AA@ 00012a2c     sgx_render_flip_test.obj
 0001:00001a40       ??_C@_0CN@CJJNALAI@Attempt?5to?5create?5transfer?5conte@ 00012a40     sgx_render_flip_test.obj
 0001:00001a70       ??_C@_0DE@BODOPOHG@Display?5Class?5API?3?5get?5the?5syste@ 00012a70     sgx_render_flip_test.obj
 0001:00001aa4       ??_C@_0CP@IFAFGPME@Display?5Class?5API?3?5map?5display?5s@ 00012aa4     sgx_render_flip_test.obj
 0001:00001ad4       ??_C@_0CH@OEGFABBA@Display?5Class?5API?3?5Map?5backbuffe@ 00012ad4     sgx_render_flip_test.obj
 0001:00001afc       ??_C@_0CF@DKIIFOJJ@Colour?5swap?5buffer?5?$CFlu?5?$CIsize?50x?$CF@ 00012afc     sgx_render_flip_test.obj
 0001:00001b24       ??_C@_0CH@MMEMFMIK@Display?5Class?5API?3?5Get?5DC?5backbu@ 00012b24     sgx_render_flip_test.obj
 0001:00001b4c       ??_C@_0DA@KBCDKOAI@Unable?5to?5create?5Display?5Class?5f@ 00012b4c     sgx_render_flip_test.obj
 0001:00001b7c       ??_C@_0DC@KJPNKNPB@Consider?5disabling?5flipping?5usin@ 00012b7c     sgx_render_flip_test.obj
 0001:00001bb0       ??_C@_0CJ@DPAIDELD@Display?5Class?5API?3?5Create?5DC?5swa@ 00012bb0     sgx_render_flip_test.obj
 0001:00001bdc       ??_C@_0DE@PBNHKLOP@Display?5Class?5API?3?5ERROR?5unsuppo@ 00012bdc     sgx_render_flip_test.obj
 0001:00001c10       ??_C@_0DH@PPPHAACG@?9?9?9?9?9?9?9?9?9?9?9?9?9?9?9?9?9?9?9?9?9?9?9?5Start?5?9?9@ 00012c10     sgx_render_flip_test.obj
 0001:00001f90       ??_C@_1EI@KHNCANBJ@?$AAF?$AAa?$AAi?$AAl?$AAe?$AAd?$AA?5?$AAt?$AAo?$AA?5?$AAc?$AAr?$AAe?$AAa?$AAt?$AAe?$AA?5?$AAt?$AAh?$AAe?$AA?5?$AAd?$AAe?$AAv?$AAi?$AAc?$AAe?$AA?5?$AAc?$AAo?$AAn?$AAt@ 00012f90     wince_unittests.obj
 0001:00001fd8       ??_C@_1BO@KHIAJBLA@?$AAI?$AAn?$AAi?$AAt?$AAi?$AAa?$AAl?$AAi?$AAz?$AAa?$AAt?$AAi?$AAo?$AAn?$AA?$AA@ 00012fd8     wince_unittests.obj
 0001:00001ff8       ??_C@_1EI@HEMGLDEE@?$AAF?$AAa?$AAi?$AAl?$AAe?$AAd?$AA?5?$AAt?$AAo?$AA?5?$AAr?$AAe?$AAg?$AAi?$AAs?$AAt?$AAe?$AAr?$AA?5?$AAt?$AAh?$AAe?$AA?5?$AAw?$AAi?$AAn?$AAd?$AAo?$AAw?$AA?5?$AAc?$AAl@ 00012ff8     wince_unittests.obj
 0001:00002040       ??_C@_1BM@GPEKOMLI@?$AAP?$AAV?$AAR?$AAS?$AAh?$AAe?$AAl?$AAl?$AAC?$AAl?$AAa?$AAs?$AAs?$AA?$AA@ 00013040     wince_unittests.obj
 0001:0000205c       ??_C@_07CHIKDHJG@?9height?$AA@ 0001305c     wince_unittests.obj
 0001:00002064       ??_C@_06EGEBBOP@?9width?$AA@ 00013064     wince_unittests.obj
 0001:0000206c       ??_C@_05MHNCFLJI@?9posy?$AA@ 0001306c     wince_unittests.obj
 0001:00002074       ??_C@_05NOMJGKNJ@?9posx?$AA@ 00013074     wince_unittests.obj
 0001:00002080       ??_C@_1KE@BDGMONOJ@?$AAH?$AA?3?$AA?2?$AAW?$AAI?$AAN?$AAC?$AAE?$AA6?$AA0?$AA0?$AA?2?$AAP?$AAL?$AAA?$AAT?$AAF?$AAO?$AAR?$AAM?$AA?2?$AAS?$AAM?$AAD?$AAK?$AAV?$AA2?$AA1?$AA0?$AA?2?$AAS?$AAR@ 00013080     wince_unittests.obj
 0001:00002124       ??_C@_1CI@OHCJFJPM@?$AAE?$AAR?$AAR?$AAO?$AAR?$AA?3?$AA?5?$AA?$CF?$AAs?$AA?5?$AAl?$AAi?$AAn?$AAe?$AA?5?$AA?$CF?$AAd?$AA?3?$AA?5?$AA?$AA@ 00013124     wince_unittests.obj
 0001:0000214c       ??_C@_1CK@MPGKAOE@?$AA?$CI?$AAe?$AAr?$AAr?$AAo?$AAr?$AA?5?$AAc?$AAo?$AAd?$AAe?$AA?3?$AA?5?$AA?$CF?$AAd?$AA?$CJ?$AA?3?$AA?5?$AA?$CF?$AAs?$AA?$AA@ 0001314c     wince_unittests.obj
 0001:00002178       ??_C@_1M@DMCDIEDK@?$AAP?$AAK?$AAM?$AA1?$AA?3?$AA?$AA@ 00013178     wince_unittests.obj
 0001:00002184       ??_C@_0L@GPAGIAIC@?9disablepm?$AA@ 00013184     wince_unittests.obj
 0001:00002190       ??_C@_1M@ILHOPKA@?$AAE?$AAr?$AAr?$AAo?$AAr?$AA?$AA@ 00013190     wince_unittests.obj
 0001:0000219c       ??_C@_1DG@PCJNAHOH@?$AAF?$AAa?$AAi?$AAl?$AAe?$AAd?$AA?5?$AAt?$AAo?$AA?5?$AAg?$AAe?$AAt?$AA?5?$AAm?$AAo?$AAn?$AAi?$AAt?$AAo?$AAr?$AA?5?$AAi?$AAn?$AAf?$AAo?$AA?$AA@ 0001319c     wince_unittests.obj
 0001:000021d4       ??_C@_07FBLHGNAH@app?4exe?$AA@ 000131d4     wince_unittests.obj
 0001:000021dc       ??_C@_0BD@FOHFKAOE@INVALID?5ERROR?5CODE?$AA@ 000131dc     sgx_unittest_utils.obj
 0001:000021f0       ??_C@_09KMCHPOPM@PVRSRV_OK?$AA@ 000131f0     sgx_unittest_utils.obj
 0001:000021fc       ??_C@_0BF@KHEAJDEG@PVRSRV_ERROR_GENERIC?$AA@ 000131fc     sgx_unittest_utils.obj
 0001:00002214       ??_C@_0BL@BOENCAIM@PVRSRV_ERROR_OUT_OF_MEMORY?$AA@ 00013214     sgx_unittest_utils.obj
 0001:00002230       ??_C@_0BN@IHBDMIPO@PVRSRV_ERROR_TOO_FEW_BUFFERS?$AA@ 00013230     sgx_unittest_utils.obj
 0001:00002250       ??_C@_0BO@EGNEIFEA@PVRSRV_ERROR_SYMBOL_NOT_FOUND?$AA@ 00013250     sgx_unittest_utils.obj
 0001:00002270       ??_C@_0BL@BKMGFOLH@PVRSRV_ERROR_OUT_OF_HSPACE?$AA@ 00013270     sgx_unittest_utils.obj
 0001:0000228c       ??_C@_0BM@LGNAOM@PVRSRV_ERROR_INVALID_PARAMS?$AA@ 0001328c     sgx_unittest_utils.obj
 0001:000022a8       ??_C@_0BN@MGJEIKFE@PVRSRV_ERROR_TILE_MAP_FAILED?$AA@ 000132a8     sgx_unittest_utils.obj
 0001:000022c8       ??_C@_0BK@JHPIKHJG@PVRSRV_ERROR_INIT_FAILURE?$AA@ 000132c8     sgx_unittest_utils.obj
 0001:000022e4       ??_C@_0CE@POPMCOCG@PVRSRV_ERROR_CANT_REGISTER_CALLB@ 000132e4     sgx_unittest_utils.obj
 0001:00002308       ??_C@_0BM@COIEDMNF@PVRSRV_ERROR_INVALID_DEVICE?$AA@ 00013308     sgx_unittest_utils.obj
 0001:00002324       ??_C@_0BH@OEOFFCIM@PVRSRV_ERROR_NOT_OWNER?$AA@ 00013324     sgx_unittest_utils.obj
 0001:0000233c       ??_C@_0BJ@PHFCJIBD@PVRSRV_ERROR_BAD_MAPPING?$AA@ 0001333c     sgx_unittest_utils.obj
 0001:00002358       ??_C@_0BF@KGIMOMJE@PVRSRV_ERROR_TIMEOUT?$AA@ 00013358     sgx_unittest_utils.obj
 0001:00002370       ??_C@_0BI@CDPBDDFH@PVRSRV_ERROR_NO_PRIMARY?$AA@ 00013370     sgx_unittest_utils.obj
 0001:00002388       ??_C@_0BP@FMELGOJO@PVRSRV_ERROR_FLIP_CHAIN_EXISTS?$AA@ 00013388     sgx_unittest_utils.obj
 0001:000023a8       ??_C@_0BN@JMHJCLJP@ERROR_CANNOT_ACQUIRE_SYSDATA?$AA@ 000133a8     sgx_unittest_utils.obj
 0001:000023c8       ??_C@_0BL@JPEIBKNH@PVRSRV_ERROR_SCENE_INVALID?$AA@ 000133c8     sgx_unittest_utils.obj
 0001:000023e4       ??_C@_0BK@JAAFMMBM@PVRSRV_ERROR_STREAM_ERROR?$AA@ 000133e4     sgx_unittest_utils.obj
 0001:00002400       ??_C@_0BP@LELIGCIL@PVRSRV_ERROR_INVALID_INTERRUPT?$AA@ 00013400     sgx_unittest_utils.obj
 0001:00002420       ??_C@_0CB@HFGDLHLE@PVRSRV_ERROR_FAILED_DEPENDENCIES@ 00013420     sgx_unittest_utils.obj
 0001:00002444       ??_C@_0BP@PFBLKCEO@PVRSRV_ERROR_CMD_NOT_PROCESSED?$AA@ 00013444     sgx_unittest_utils.obj
 0001:00002464       ??_C@_0BJ@PHLIKBPN@PVRSRV_ERROR_CMD_TOO_BIG?$AA@ 00013464     sgx_unittest_utils.obj
 0001:00002480       ??_C@_0CE@FHHHLEGE@PVRSRV_ERROR_DEVICE_REGISTER_FAI@ 00013480     sgx_unittest_utils.obj
 0001:000024a4       ??_C@_0BI@JBKNPCOM@PVRSRV_ERROR_FIFO_SPACE?$AA@ 000134a4     sgx_unittest_utils.obj
 0001:000024bc       ??_C@_0BJ@IIGHNIEG@PVRSRV_ERROR_TA_RECOVERY?$AA@ 000134bc     sgx_unittest_utils.obj
 0001:000024d8       ??_C@_0BN@BKNBJNB@PVRSRV_ERROR_INDOSORLOWPOWER?$AA@ 000134d8     sgx_unittest_utils.obj
 0001:000024f8       ??_C@_0BM@MCHBLHIP@PVRSRV_ERROR_TOOMANYBUFFERS?$AA@ 000134f8     sgx_unittest_utils.obj
 0001:00002514       ??_C@_0BL@FINKNLDE@PVRSRV_ERROR_NOT_SUPPORTED?$AA@ 00013514     sgx_unittest_utils.obj
 0001:00002530       ??_C@_0CA@KIDKOOGL@PVRSRV_ERROR_PROCESSING_BLOCKED?$AA@ 00013530     sgx_unittest_utils.obj
 0001:00002550       ??_C@_0BG@OJDNODAO@PVRSRV_ERROR_NO_MUTEX?$AA@ 00013550     sgx_unittest_utils.obj
 0001:00002568       ??_C@_0CA@NBGAMPKE@PVRSRV_ERROR_CANNOT_FLUSH_QUEUE?$AA@ 00013568     sgx_unittest_utils.obj
 0001:00002588       ??_C@_0CE@NLLBGAEA@PVRSRV_ERROR_CANNOT_GET_QUEUE_SP@ 00013588     sgx_unittest_utils.obj
 0001:000025ac       ??_C@_0CG@FCILKACH@PVRSRV_ERROR_CANNOT_GET_RENDERDE@ 000135ac     sgx_unittest_utils.obj
 0001:000025d4       ??_C@_0BD@COEEPPOL@PVRSRV_ERROR_RETRY?$AA@ 000135d4     sgx_unittest_utils.obj
 0001:000025e8       ??_C@_04LNELOFCG@?5OK?6?$AA@ 000135e8     sgx_unittest_utils.obj
 0001:000025f0       ??_C@_0BB@EIDKNEMM@?5FAIL?5?9?5?$CFs?$CI?$CFlu?$CJ?6?$AA@ 000135f0     sgx_unittest_utils.obj
 0001:00002604       ??_C@_0CD@KNHKMALC@Unknown?5option?5?$CFs?6Use?5?9h?5for?5hel@ 00013604     sgx_unittest_utils.obj
 0001:00002628       ??_C@_09KDMOKIPB@?$CFs?5?$CFs?7?$CFs?6?$AA@ 00013628     sgx_unittest_utils.obj
 0001:00002634       ??_C@_0N@BINAGECB@?$CFs?5options?3?6?$AA@ 00013634     sgx_unittest_utils.obj
 0001:00002644       ??_C@_02JNAPBCPB@?9h?$AA@  00013644     sgx_unittest_utils.obj
 0001:00002648       ??_C@_0DA@BEOOOKFN@?$CFs?5?$CI?$CFlu?$CJ?0?5write?5ops?5complete?3?5?$CFl@ 00013648     sgx_unittest_utils.obj
 0001:00002678       ??_C@_0BJ@IMBALOKG@PVRSRV_DEVICE_ID_UNKNOWN?$AA@ 00013678     sgx_unittest_utils.obj
 0001:00002694       ??_C@_0BH@OGEGGGCD@PVRSRV_DEVICE_ID_MSVDX?$AA@ 00013694     sgx_unittest_utils.obj
 0001:000026ac       ??_C@_0BF@BBCLGMON@PVRSRV_DEVICE_ID_SGX?$AA@ 000136ac     sgx_unittest_utils.obj
 0001:000026c4       ??_C@_0CD@BDGFMHBG@PVRSRV_DEVICE_TYPE_EXT?5?$CI3rd?5Part@ 000136c4     sgx_unittest_utils.obj
 0001:000026e8       ??_C@_0BE@GEDKFGMC@Not?5recognised?50x?$CFx?$AA@ 000136e8     sgx_unittest_utils.obj
 0001:000026fc       ??_C@_0BI@ICLDLMDM@?4?4?4?4?5ui32ProcessID?3?$CFlu?6?$AA@ 000136fc     sgx_unittest_utils.obj
 0001:00002718       ??_C@_0EK@BPNJOJAB@?4?4?4?4?5Shared?5heap?5?$CFlu?5?9?5HeapID?30x@ 00013718     sgx_unittest_utils.obj
 0001:00002764       ??_C@_0CL@DNLHEBLI@Attempt?5to?5create?5memory?5context@ 00013764     sgx_unittest_utils.obj
 0001:00002790       ??_C@_0ED@NNKEOJPF@?4?4?4?4?5Display?5dimensions?5?$CFlu?5?9?5By@ 00013790     sgx_unittest_utils.obj
 0001:000027d4       ??_C@_0DB@DPDHNDGF@Display?5Class?5API?3?5enumerate?5dis@ 000137d4     sgx_unittest_utils.obj
 0001:00002808       ??_C@_0CK@PAKBMFJN@?4?4?4?4?5Display?5format?5?$CFlu?5?9?5Pixelf@ 00013808     sgx_unittest_utils.obj
 0001:00002834       ??_C@_0CF@FMDFFMKC@Display?5Class?5API?3?5Get?5display?5i@ 00013834     sgx_unittest_utils.obj
 0001:0000285c       ??_C@_0O@GDPIEJBG@?4?4?4?4?5Name?3?$CFs?6?$AA@ 0001385c     sgx_unittest_utils.obj
 0001:0000286c       ??_C@_0BI@BLGHILNJ@?4?4?4?4?5MaxSwapChains?3?$CFlu?6?$AA@ 0001386c     sgx_unittest_utils.obj
 0001:00002884       ??_C@_0BO@POAFDAJE@?4?4?4?4?5MaxSwapChainBuffers?3?$CFlu?6?$AA@ 00013884     sgx_unittest_utils.obj
 0001:000028a4       ??_C@_0BK@CPCAOBID@?4?4?4?4?5MinSwapInterval?3?$CFlu?6?$AA@ 000138a4     sgx_unittest_utils.obj
 0001:000028c0       ??_C@_0BK@DMGFAHCI@?4?4?4?4?5MaxSwapInterval?3?$CFlu?6?$AA@ 000138c0     sgx_unittest_utils.obj
 0001:000028dc       ??_C@_0CO@GIPBIACE@Display?5Class?5API?3?5enumerate?5dis@ 000138dc     sgx_unittest_utils.obj
 0001:0000290c       ??_C@_0CA@DAONOMAK@Display?5Class?5API?3?5open?5device?6?$AA@ 0001390c     sgx_unittest_utils.obj
 0001:0000292c       ??_C@_0CG@MMBLEMBO@Display?5Class?5API?3?5enumerate?5dev@ 0001392c     sgx_unittest_utils.obj
 0001:00002954       ??_C@_0DM@CIPNLPOO@PVRSRVEnumerateDeviceClass?$CI?$CJ?5ret@ 00013954     sgx_unittest_utils.obj
 0001:00002990       ??_C@_0BJ@NLALCGOE@Getting?5SGX?5Client?5info?6?$AA@ 00013990     sgx_unittest_utils.obj
 0001:000029ac       ??_C@_0BP@IDIGABKI@Attempt?5to?5acquire?5device?5?$CFd?3?6?$AA@ 000139ac     sgx_unittest_utils.obj
 0001:000029cc       ??_C@_0BH@PPGIPGOP@?5?5?5?5?5?5?5?5?5?5?5?5?$CF04d?5?5?5?5?$HM?5?$AA@ 000139cc     sgx_unittest_utils.obj
 0001:000029e4       ??_C@_0CL@KFFMIBHA@Call?5PVRSRVConnect?5with?5a?5valid?5@ 000139e4     sgx_unittest_utils.obj
 0001:00002a10       ??_C@_0DE@KAFOOJDI@Get?5number?5of?5devices?5from?5PVRSR@ 00013a10     sgx_unittest_utils.obj
 0001:00002a44       ??_C@_0BK@GEDDINJE@?4?4?4?4?5Reported?5?$CFu?5devices?6?$AA@ 00013a44     sgx_unittest_utils.obj
 0001:00002a60       ??_C@_0CD@INKLJIDI@?4?4?4?4?5Device?5Number?5?5?$HM?5Device?5Typ@ 00013a60     sgx_unittest_utils.obj
 0001:00002a84       ??_C@_0BP@HJNHLLEN@Destroy?5Device?5Memory?5Context?6?$AA@ 00013a84     sgx_unittest_utils.obj
 0001:00002aa4       ??_C@_0CF@DBFHMBAF@Display?5Class?5API?3?5close?5the?5dev@ 00013aa4     sgx_unittest_utils.obj
 0001:00002acc       ??_C@_0BK@HGIBJBNI@Release?5SGX?5Client?5Info?3?6?$AA@ 00013acc     sgx_unittest_utils.obj
 0001:00002ae8       ??_C@_0BL@JBOAKENO@Disconnect?5from?5services?3?6?$AA@ 00013ae8     sgx_unittest_utils.obj
 0001:00002b38       srft_EncodeDmaBurst        00013b38 f   sgx_render_flip_test.obj
 0001:00006bf0       main                       00017bf0 f   sgx_render_flip_test.obj
 0001:0000752c       PDSGeneratePixelEventProgram 0001852c f   pds.obj
 0001:000076d0       PDSGeneratePixelShaderSAProgram 000186d0 f   pds.obj
 0001:00007978       PDSGeneratePixelShaderProgram 00018978 f   pds.obj
 0001:00007bc8       PDSGenerateStateCopyProgram 00018bc8 f   pds.obj
 0001:00007d38       PDSGenerateVertexShaderProgram 00018d38 f   pds.obj
 0001:00008404       PDSGenerateTerminateStateProgram 00019404 f   pds.obj
 0001:000084ac       WriteEndOfPassUSSECode     000194ac f   pixevent.obj
 0001:000084c4       WriteEndOfRenderUSSECode   000194c4 f   pixevent.obj
 0001:000084f4       WriteEndOfTileUSSECode     000194f4 f   pixevent.obj
 0001:000085b4       AppWndProc                 000195b4 f   wince_unittests.obj
 0001:00008614       WinMain                    00019614 f   wince_unittests.obj
 0001:00008b50       sgxut_GetErrorString       00019b50 f   sgx_unittest_utils.obj
 0001:00008d24       sgxut_null_dpf             00019d24 f   sgx_unittest_utils.obj
 0001:00008d38       sgxut_fail_if_error        00019d38 f   sgx_unittest_utils.obj
 0001:00008d74       sgxut_fail_if_error_quiet  00019d74 f   sgx_unittest_utils.obj
 0001:00008da4       sgxut_parse_commandline_option 00019da4 f   sgx_unittest_utils.obj
 0001:00008e78       sgxut_sleep_ms             00019e78 f   sgx_unittest_utils.obj
 0001:00008e7c       sgxut_sleep_us             00019e7c f   sgx_unittest_utils.obj
 0001:00008e80       sgxut_wait_for_buffer      00019e80 f   sgx_unittest_utils.obj
 0001:00008f18       sgxut_get_current_time     00019f18 f   sgx_unittest_utils.obj
 0001:00008f74       sgxut_print_dev_type       00019f74 f   sgx_unittest_utils.obj
 0001:00008fd4       sgxut_SGXInit              00019fd4 f   sgx_unittest_utils.obj
 0001:000095b8       sgxut_SGXDeInit            0001a5b8 f   sgx_unittest_utils.obj
 0001:00009678       SGXQueueTransfer           0001a678 f   srvclum:SRVCLUM.dll
 0001:00009688       SGXAddRenderTarget         0001a688 f   srvclum:SRVCLUM.dll
 0001:00009698       SGXRemoveRenderTarget      0001a698 f   srvclum:SRVCLUM.dll
 0001:000096a8       PVRSRVSwapToDCBuffer       0001a6a8 f   srvclum:SRVCLUM.dll
 0001:000096b8       SGXKickTA                  0001a6b8 f   srvclum:SRVCLUM.dll
 0001:000096c8       PVRSRVFreeDeviceMem        0001a6c8 f   srvclum:SRVCLUM.dll
 0001:000096d8       PVRSRVAllocDeviceMem       0001a6d8 f   srvclum:SRVCLUM.dll
 0001:000096e8       PVRSRVDestroyDCSwapChain   0001a6e8 f   srvclum:SRVCLUM.dll
 0001:000096f8       PVRSRVUnmapDeviceClassMemory 0001a6f8 f   srvclum:SRVCLUM.dll
 0001:00009708       SGXDestroyTransferContext  0001a708 f   srvclum:SRVCLUM.dll
 0001:00009718       SGXDestroyRenderContext    0001a718 f   srvclum:SRVCLUM.dll
 0001:00009728       SGXSetContextPriority      0001a728 f   srvclum:SRVCLUM.dll
 0001:00009738       SGXCreateRenderContext     0001a738 f   srvclum:SRVCLUM.dll
 0001:00009748       PVRSRVGetMiscInfo          0001a748 f   srvclum:SRVCLUM.dll
 0001:00009758       PVRSRVGetDCSystemBuffer    0001a758 f   srvclum:SRVCLUM.dll
 0001:00009768       SGXCreateTransferContext   0001a768 f   srvclum:SRVCLUM.dll
 0001:00009778       PVRSRVMapDeviceClassMemory 0001a778 f   srvclum:SRVCLUM.dll
 0001:00009788       PVRSRVGetDCBuffers         0001a788 f   srvclum:SRVCLUM.dll
 0001:00009798       PVRSRVCreateDCSwapChain    0001a798 f   srvclum:SRVCLUM.dll
 0001:000097a8       PVRSRVWaitus               0001a7a8 f   srvclum:SRVCLUM.dll
 0001:000097b8       PVRSRVEventObjectWait      0001a7b8 f   srvclum:SRVCLUM.dll
 0001:000097c8       PVRSRVCreateDeviceMemContext 0001a7c8 f   srvclum:SRVCLUM.dll
 0001:000097d8       PVRSRVEnumDCDims           0001a7d8 f   srvclum:SRVCLUM.dll
 0001:000097e8       PVRSRVEnumDCFormats        0001a7e8 f   srvclum:SRVCLUM.dll
 0001:000097f8       PVRSRVGetDCInfo            0001a7f8 f   srvclum:SRVCLUM.dll
 0001:00009808       PVRSRVOpenDCDevice         0001a808 f   srvclum:SRVCLUM.dll
 0001:00009818       PVRSRVEnumerateDeviceClass 0001a818 f   srvclum:SRVCLUM.dll
 0001:00009828       SGXGetClientInfo           0001a828 f   srvclum:SRVCLUM.dll
 0001:00009838       PVRSRVAcquireDeviceData    0001a838 f   srvclum:SRVCLUM.dll
 0001:00009848       PVRSRVEnumerateDevices     0001a848 f   srvclum:SRVCLUM.dll
 0001:00009858       PVRSRVConnect              0001a858 f   srvclum:SRVCLUM.dll
 0001:00009868       PVRSRVDisconnect           0001a868 f   srvclum:SRVCLUM.dll
 0001:00009878       SGXReleaseClientInfo       0001a878 f   srvclum:SRVCLUM.dll
 0001:00009888       PVRSRVCloseDCDevice        0001a888 f   srvclum:SRVCLUM.dll
 0001:00009898       PVRSRVDestroyDeviceMemContext 0001a898 f   srvclum:SRVCLUM.dll
 0001:000098a8       PostQuitMessage            0001a8a8 f   coredll:COREDLL.dll
 0001:000098b8       DefWindowProcW             0001a8b8 f   coredll:COREDLL.dll
 0001:000098c8       ReleasePowerRequirement    0001a8c8 f   coredll:COREDLL.dll
 0001:000098d8       DestroyWindow              0001a8d8 f   coredll:COREDLL.dll
 0001:000098e8       ReleaseDC                  0001a8e8 f   coredll:COREDLL.dll
 0001:000098f8       GetDC                      0001a8f8 f   coredll:COREDLL.dll
 0001:00009908       CreateWindowExW            0001a908 f   coredll:COREDLL.dll
 0001:00009918       RegisterClassW             0001a918 f   coredll:COREDLL.dll
 0001:00009928       GetStockObject             0001a928 f   coredll:COREDLL.dll
 0001:00009938       NKDbgPrintfW               0001a938 f   coredll:COREDLL.dll
 0001:00009948       FormatMessageW             0001a948 f   coredll:COREDLL.dll
 0001:00009958       GetLastError               0001a958 f   coredll:COREDLL.dll
 0001:00009968       SetPowerRequirement        0001a968 f   coredll:COREDLL.dll
 0001:00009978       WideCharToMultiByte        0001a978 f   coredll:COREDLL.dll
 0001:00009988       SetCursorPos               0001a988 f   coredll:COREDLL.dll
 0001:00009998       GetCursorPos               0001a998 f   coredll:COREDLL.dll
 0001:000099a8       MessageBoxW                0001a9a8 f   coredll:COREDLL.dll
 0001:000099b8       GetMonitorInfo             0001a9b8 f   coredll:COREDLL.dll
 0001:000099c8       MonitorFromPoint           0001a9c8 f   coredll:COREDLL.dll
 0001:000099d8       GetSystemMetrics           0001a9d8 f   coredll:COREDLL.dll
 0001:000099e8       Sleep                      0001a9e8 f   coredll:COREDLL.dll
 0001:000099f8       QueryPerformanceFrequency  0001a9f8 f   coredll:COREDLL.dll
 0001:00009a08       QueryPerformanceCounter    0001aa08 f   coredll:COREDLL.dll
 0001:00009a98       WinMainCRTStartup          0001aa98 f   corelib0:pegwmain.obj
 0001:00009acc       __GSHandlerCheckCommon     0001aacc f   corelib0:gshandler.obj
 0001:00009b08       __GSHandlerCheck           0001ab08 f   corelib0:gshandler.obj
 0001:00009b2c       __security_init_cookie     0001ab2c f   corelib0:seccinit.obj
 0001:00009b88       __security_check_cookie    0001ab88 f   corelib0:armsecgs.obj
 0001:00009b9c       __gsfailure                0001ab9c f   corelib0:armsecgs.obj
 0001:00009ca8       exit                       0001aca8 f   corelib0:cexit.obj
 0001:00009cc0       _exit                      0001acc0 f   corelib0:cexit.obj
 0001:00009d00       _initterm                  0001ad00 f   corelib0:crt0dat.obj
 0001:00009d34       _cinit                     0001ad34 f   corelib0:crt0dat.obj
 0001:00009d68       printf                     0001ad68 f   corelib1:COREDLL.dll
 0001:00009d78       memset                     0001ad78 f   corelib1:COREDLL.dll
 0001:00009d88       free                       0001ad88 f   corelib1:COREDLL.dll
 0001:00009d98       getchar                    0001ad98 f   corelib1:COREDLL.dll
 0001:00009da8       malloc                     0001ada8 f   corelib1:COREDLL.dll
 0001:00009db8       sprintf                    0001adb8 f   corelib1:COREDLL.dll
 0001:00009dc8       memcpy                     0001adc8 f   corelib1:COREDLL.dll
 0001:00009dd8       strtol                     0001add8 f   corelib1:COREDLL.dll
 0001:00009de8       atol                       0001ade8 f   corelib1:COREDLL.dll
 0001:00009df8       strcmp                     0001adf8 f   corelib1:COREDLL.dll
 0001:00009e08       atoi                       0001ae08 f   corelib1:COREDLL.dll
 0001:00009e18       _stricmp                   0001ae18 f   corelib1:COREDLL.dll
 0001:00009e28       _isctype                   0001ae28 f   corelib1:COREDLL.dll
 0001:00009e38       wcslen                     0001ae38 f   corelib1:COREDLL.dll
 0001:00009e48       _XcptFilter                0001ae48 f   corelib1:COREDLL.dll
 0001:00009e58       __C_specific_handler       0001ae58 f   corelib1:COREDLL.dll
 0001:00009e68       __security_gen_cookie2     0001ae68 f   corelib1:COREDLL.dll
 0001:00009e78       __report_gsfailure         0001ae78 f   corelib1:COREDLL.dll
 0001:00009e88       TerminateProcess           0001ae88 f   coredll:COREDLL.dll
 0001:00009eb8       __IMPORT_DESCRIPTOR_SRVCLUM 0001aeb8     srvclum:SRVCLUM.dll
 0001:00009ecc       __IMPORT_DESCRIPTOR_COREDLL 0001aecc     coredll:COREDLL.dll
 0001:00009ee0       __NULL_IMPORT_DESCRIPTOR   0001aee0     srvclum:SRVCLUM.dll
 0002:00000000       __imp_GetLastError         0001c000     coredll:COREDLL.dll
 0002:00000004       __imp___report_gsfailure   0001c004     corelib1:COREDLL.dll
 0002:00000008       __imp___security_gen_cookie2 0001c008     corelib1:COREDLL.dll
 0002:0000000c       __imp___C_specific_handler 0001c00c     corelib1:COREDLL.dll
 0002:00000010       __imp__XcptFilter          0001c010     corelib1:COREDLL.dll
 0002:00000014       __imp___rt_sdiv64by64      0001c014     corelib1:COREDLL.dll
 0002:00000018       __imp_wcslen               0001c018     corelib1:COREDLL.dll
 0002:0000001c       __imp__isctype             0001c01c     corelib1:COREDLL.dll
 0002:00000020       __imp__stricmp             0001c020     corelib1:COREDLL.dll
 0002:00000024       __imp_atoi                 0001c024     corelib1:COREDLL.dll
 0002:00000028       __imp_strcmp               0001c028     corelib1:COREDLL.dll
 0002:0000002c       __imp_atol                 0001c02c     corelib1:COREDLL.dll
 0002:00000030       __imp_strtol               0001c030     corelib1:COREDLL.dll
 0002:00000034       __imp_memcpy               0001c034     corelib1:COREDLL.dll
 0002:00000038       __imp_sprintf              0001c038     corelib1:COREDLL.dll
 0002:0000003c       __imp_malloc               0001c03c     corelib1:COREDLL.dll
 0002:00000040       __imp_getchar              0001c040     corelib1:COREDLL.dll
 0002:00000044       __imp_free                 0001c044     corelib1:COREDLL.dll
 0002:00000048       __imp_memset               0001c048     corelib1:COREDLL.dll
 0002:0000004c       __imp___dtos               0001c04c     corelib1:COREDLL.dll
 0002:00000050       __imp_sin                  0001c050     corelib1:COREDLL.dll
 0002:00000054       __imp___stod               0001c054     corelib1:COREDLL.dll
 0002:00000058       __imp_cos                  0001c058     corelib1:COREDLL.dll
 0002:0000005c       __imp___lts                0001c05c     corelib1:COREDLL.dll
 0002:00000060       __imp___gts                0001c060     corelib1:COREDLL.dll
 0002:00000064       __imp___negs               0001c064     corelib1:COREDLL.dll
 0002:00000068       __imp___divs               0001c068     corelib1:COREDLL.dll
 0002:0000006c       __imp___stou               0001c06c     corelib1:COREDLL.dll
 0002:00000070       __imp___adds               0001c070     corelib1:COREDLL.dll
 0002:00000074       __imp___muls               0001c074     corelib1:COREDLL.dll
 0002:00000078       __imp___utos               0001c078     corelib1:COREDLL.dll
 0002:0000007c       __imp___subs               0001c07c     corelib1:COREDLL.dll
 0002:00000080       __imp_printf               0001c080     corelib1:COREDLL.dll
 0002:00000084       __imp_PostQuitMessage      0001c084     coredll:COREDLL.dll
 0002:00000088       __imp_DefWindowProcW       0001c088     coredll:COREDLL.dll
 0002:0000008c       __imp_ReleasePowerRequirement 0001c08c     coredll:COREDLL.dll
 0002:00000090       __imp_DestroyWindow        0001c090     coredll:COREDLL.dll
 0002:00000094       __imp_ReleaseDC            0001c094     coredll:COREDLL.dll
 0002:00000098       __imp_GetDC                0001c098     coredll:COREDLL.dll
 0002:0000009c       __imp_CreateWindowExW      0001c09c     coredll:COREDLL.dll
 0002:000000a0       __imp_RegisterClassW       0001c0a0     coredll:COREDLL.dll
 0002:000000a4       __imp_GetStockObject       0001c0a4     coredll:COREDLL.dll
 0002:000000a8       __imp_NKDbgPrintfW         0001c0a8     coredll:COREDLL.dll
 0002:000000ac       __imp_FormatMessageW       0001c0ac     coredll:COREDLL.dll
 0002:000000b0       __imp_TerminateProcess     0001c0b0     coredll:COREDLL.dll
 0002:000000b4       __imp_SetPowerRequirement  0001c0b4     coredll:COREDLL.dll
 0002:000000b8       __imp_WideCharToMultiByte  0001c0b8     coredll:COREDLL.dll
 0002:000000bc       __imp_SetCursorPos         0001c0bc     coredll:COREDLL.dll
 0002:000000c0       __imp_GetCursorPos         0001c0c0     coredll:COREDLL.dll
 0002:000000c4       __imp_MessageBoxW          0001c0c4     coredll:COREDLL.dll
 0002:000000c8       __imp_GetMonitorInfo       0001c0c8     coredll:COREDLL.dll
 0002:000000cc       __imp_MonitorFromPoint     0001c0cc     coredll:COREDLL.dll
 0002:000000d0       __imp_GetSystemMetrics     0001c0d0     coredll:COREDLL.dll
 0002:000000d4       __imp_Sleep                0001c0d4     coredll:COREDLL.dll
 0002:000000d8       __imp_QueryPerformanceFrequency 0001c0d8     coredll:COREDLL.dll
 0002:000000dc       __imp_QueryPerformanceCounter 0001c0dc     coredll:COREDLL.dll
 0002:000000e0       __imp___rt_udiv            0001c0e0     corelib1:COREDLL.dll
 0002:000000e4       \177COREDLL_NULL_THUNK_DATA 0001c0e4     coredll:COREDLL.dll
 0002:000000e8       __imp_PVRSRVDestroyDeviceMemContext 0001c0e8     srvclum:SRVCLUM.dll
 0002:000000ec       __imp_PVRSRVCloseDCDevice  0001c0ec     srvclum:SRVCLUM.dll
 0002:000000f0       __imp_SGXReleaseClientInfo 0001c0f0     srvclum:SRVCLUM.dll
 0002:000000f4       __imp_PVRSRVDisconnect     0001c0f4     srvclum:SRVCLUM.dll
 0002:000000f8       __imp_PVRSRVConnect        0001c0f8     srvclum:SRVCLUM.dll
 0002:000000fc       __imp_PVRSRVEnumerateDevices 0001c0fc     srvclum:SRVCLUM.dll
 0002:00000100       __imp_PVRSRVAcquireDeviceData 0001c100     srvclum:SRVCLUM.dll
 0002:00000104       __imp_SGXGetClientInfo     0001c104     srvclum:SRVCLUM.dll
 0002:00000108       __imp_PVRSRVEnumerateDeviceClass 0001c108     srvclum:SRVCLUM.dll
 0002:0000010c       __imp_PVRSRVOpenDCDevice   0001c10c     srvclum:SRVCLUM.dll
 0002:00000110       __imp_PVRSRVGetDCInfo      0001c110     srvclum:SRVCLUM.dll
 0002:00000114       __imp_PVRSRVEnumDCFormats  0001c114     srvclum:SRVCLUM.dll
 0002:00000118       __imp_PVRSRVEnumDCDims     0001c118     srvclum:SRVCLUM.dll
 0002:0000011c       __imp_PVRSRVCreateDeviceMemContext 0001c11c     srvclum:SRVCLUM.dll
 0002:00000120       __imp_PVRSRVEventObjectWait 0001c120     srvclum:SRVCLUM.dll
 0002:00000124       __imp_PVRSRVWaitus         0001c124     srvclum:SRVCLUM.dll
 0002:00000128       __imp_PVRSRVCreateDCSwapChain 0001c128     srvclum:SRVCLUM.dll
 0002:0000012c       __imp_PVRSRVGetDCBuffers   0001c12c     srvclum:SRVCLUM.dll
 0002:00000130       __imp_PVRSRVMapDeviceClassMemory 0001c130     srvclum:SRVCLUM.dll
 0002:00000134       __imp_SGXCreateTransferContext 0001c134     srvclum:SRVCLUM.dll
 0002:00000138       __imp_PVRSRVGetDCSystemBuffer 0001c138     srvclum:SRVCLUM.dll
 0002:0000013c       __imp_PVRSRVGetMiscInfo    0001c13c     srvclum:SRVCLUM.dll
 0002:00000140       __imp_SGXCreateRenderContext 0001c140     srvclum:SRVCLUM.dll
 0002:00000144       __imp_SGXSetContextPriority 0001c144     srvclum:SRVCLUM.dll
 0002:00000148       __imp_SGXDestroyRenderContext 0001c148     srvclum:SRVCLUM.dll
 0002:0000014c       __imp_SGXDestroyTransferContext 0001c14c     srvclum:SRVCLUM.dll
 0002:00000150       __imp_PVRSRVUnmapDeviceClassMemory 0001c150     srvclum:SRVCLUM.dll
 0002:00000154       __imp_PVRSRVDestroyDCSwapChain 0001c154     srvclum:SRVCLUM.dll
 0002:00000158       __imp_PVRSRVAllocDeviceMem 0001c158     srvclum:SRVCLUM.dll
 0002:0000015c       __imp_PVRSRVFreeDeviceMem  0001c15c     srvclum:SRVCLUM.dll
 0002:00000160       __imp_SGXKickTA            0001c160     srvclum:SRVCLUM.dll
 0002:00000164       __imp_PVRSRVSwapToDCBuffer 0001c164     srvclum:SRVCLUM.dll
 0002:00000168       __imp_SGXRemoveRenderTarget 0001c168     srvclum:SRVCLUM.dll
 0002:0000016c       __imp_SGXAddRenderTarget   0001c16c     srvclum:SRVCLUM.dll
 0002:00000170       __imp_SGXQueueTransfer     0001c170     srvclum:SRVCLUM.dll
 0002:00000174       \177SRVCLUM_NULL_THUNK_DATA 0001c174     srvclum:SRVCLUM.dll
 0002:0000017c       gui32WindowWidth           0001c17c     wince_unittests.obj
 0002:00000180       gui32WindowHeight          0001c180     wince_unittests.obj
 0002:00000184       gui32PosX                  0001c184     wince_unittests.obj
 0002:00000188       gui32PosY                  0001c188     wince_unittests.obj
 0002:0000018c       __security_cookie          0001c18c     corelib0:seccinit.obj
 0002:00000190       __security_cookie_complement 0001c190     corelib0:seccinit.obj
 0002:000001c4       gbWindow                   0001c1c4     wince_unittests.obj
 0002:000001c8       ghWnd                      0001c1c8     wince_unittests.obj
 0002:000001cc       pfnRegisteredWndProc       0001c1cc     wince_unittests.obj
 0002:000001d0       _exitflag                  0001c1d0     corelib0:cexit.obj
 0002:000001d4       gui32DisplayWidth          0001c1d4     <common>
 0002:000001d8       gui32DisplayHeight         0001c1d8     <common>
 0002:000001dc       __onexitend                0001c1dc     <common>
 0002:000001e0       __onexitbegin              0001c1e0     <common>

 entry point at        0001:00009a98

 Static symbols

 0001:00002be4       srft_InsertSlowDown        00013be4 f   sgx_render_flip_test.obj
 0001:00002ca4       srft_wait_for_render       00013ca4 f   sgx_render_flip_test.obj
 0001:00002da0       srft_Interpolate           00013da0 f   sgx_render_flip_test.obj
 0001:00002e64       srft_CyclePositionInterpolate 00013e64 f   sgx_render_flip_test.obj
 0001:00002f84       srft_WriteSecondaryPixelCode 00013f84 f   sgx_render_flip_test.obj
 0001:00003074       srft_WritePrimaryPixelCode 00014074 f   sgx_render_flip_test.obj
 0001:0000326c       srft_WriteMTEStateCode     0001426c f   sgx_render_flip_test.obj
 0001:0000340c       srft_WriteVerticesToVertexDataBuffer 0001440c f   sgx_render_flip_test.obj
 0001:00003cbc       srft_WriteVertexShaderCode 00014cbc f   sgx_render_flip_test.obj
 0001:00003f28       srft_SetupTAKick           00014f28 f   sgx_render_flip_test.obj
 0001:00004084       srft_PresentBlit           00015084 f   sgx_render_flip_test.obj
 0001:000041fc       srft_PerThread             000151fc f   sgx_render_flip_test.obj
 0001:00005ed8       srft_ParseOptions          00016ed8 f   sgx_render_flip_test.obj
 0001:000075cc       PDSEncodeSimpleMOVS        000185cc f   pds.obj
 0001:00007648       PDSGetNextConstant         00018648 f   pds.obj
 0001:0000768c       PDSGetNumConstants         0001868c f   pds.obj
 0001:00009a20       WinMainCRTStartupHelper    0001aa20 f   corelib0:pegwmain.obj
 0001:00009be0       doexit                     0001abe0 f   corelib0:cexit.obj
